:101DEA002020202020200D0A002A56455253494F10
:101DFA004E3A20522D4441532056322E330D0A00BA
:101E0A002A4D4553534147453A2053656C667465DC
:101E1A007374207061737365640D0A002A57415206
:101E2A004E494E473A2053656C6674657374206652
:101E3A0061696C65640D0A002A52454144590D0ACC
:101E4A0000000000002A01005202007903009E04EB
:101E5A0000C20500E5060106070127080146090137
:101E6A00640A01E90F02581403001E03742803C30D
:071E7A003203F93C04023EB3
:100CA3009070F0EEF0A3EFF0A37401F09070F2E017
:100CB300FF6412602AEF75F003A4244BF582E43439
:100CC3001EF583E493FC740193FDC39070F1E09DE2
:100CD3009070F0E09C40089070F2E004F080CDEF5B
:100CE30075F003A4244BF582E4341EF583E493FEEC
:100CF300740193FF9070F0E0FCA3E0FDC3EF9DFF50
:100D0300EE9CFEE4FCFDC8ECC8C9EDC9CAEECACB33
:100D1300EFCBA3E075F003A4244AF582E4341EF577
:100D230083E493FFE4FE1204C0ECC0E0EDC0E0EE08
:100D3300C0E0EFC0E09070F2E075F003A42448F542
:100D430082E4341EF583E493FE740193FFC3907031
:100D5300F1E09FFF9070F0E09EFEE4FCFDC8ECC85C
:100D6300C9EDC9CAEECACBEFCB9070F2E075F003C0
:100D7300A4244DF582E4341EF583E493FFE4FE12CC
:100D830004C0D0E0FBD0E0FAD0E0F9D0E0F8EF2BDC
:100D9300FFEE3AFEED39FDEC38FC9070F3120617C6
:100DA3007FE87E037D007C009070F3E0F8A3E0F918
:100DB300A3E0FAA3E0FB1204C0C8ECC8C9EDC9CA9A
:100DC300EECACBEFCB9070F2E0FF75F003A424489A
:100DD300F582E4341EF583E493FC740193FDEF750F
:100DE300F003A4244BF582E4341EF583C37401930A
:100DF3009DFFE4939CC313FEEF13FFE4FCFDEB2F75
:100E0300FFEA3EFEED39FDEC38FCECC0E0EDC0E05E
:100E1300EEC0E0EFC0E09070F2E0FF75F003A424B1
:100E230048F582E4341EF583E493FC740193FDEFEB
:100E330075F003A4244BF582E4341EF583C37401D7
:100E4300939DFFE4939CFEE4FCFDF8F9CAEECACB44
:100E5300EFCBD0E0FFD0E0FED0E0FDD0E0FC120508
:020E63004B2220
:10167900301503021716E56064036009E560640B21
:10168900600302177BC3E54E78CE96FFE54D1896A9
:10169900FE120CA3CBEFCBCAEECAEB4A7003FA7B5E
:1016A90001D201E49070E9F0CEEACECFEBCF7C0015
:1016B9007D0A1204099070E9E024EAF582E43470A5
:1016C900F583EDF0CEEACECFEBCF7C007D0A120494
:1016D90009CAEECACBEFCB9070E9E004F0E0B4059B
:1016E900C79070E97404F09070E9E0FFF460157434
:1016F900EA2FF582E43470F583E070089070E9E030
:1017090014F080E3EF049070EFF0D215227F1E12DF
:101719002BBB7F017D327B04122C933013043017CD
:10172900FA227F0A122BBB9070EFE0149070E9F057
:101739009070E9E024EAF582E43470F583E0700BF7
:101749007F017D0B7B04122C9380169070E9E024B5
:10175900EAF582E43470F583E0FF7D0B7B01122CFE
:10176900933013043017FA229070E9E0FF14F0EF78
:0317790070BE221D
:101F9800D2AF122AC9122BDE122B56122AFB122C90
:101FA800C7122C43122C871221747BFF7A1D79EA01
:101FB8001200C97BFF7A1D79F31200C912278F50CE
:101FC800107BFF7A1E790A1200C97F01122C6980E2
:101FD800097BFF7A1E79261200C91223889070A403
:101FE800E0FF12271D1229451224B19070A5E0FECA
:101FF800A3E0FF1226207BFF7A1E79421200C9C295
:0D20080015301703122AE312167980F52215
:03000B000220913F
:10209100C0E0C0F0C083C082C0D075D008C28CAF90
:1020A1008CEFFEAD8AED255778D0F6E5563E18F651
:1020B100F58C08E6F58AD28CD2C4C2C4D55B0990EE
:1020C100709BE0F55B1229D5D55A1B90709BE0F50A
:1020D1005A0559E55970020558E55945587007E503
:1020E100606003756005E5606404600C12187E127F
:1020F10023EE121BE0121E81D0D0D082D083D0F00B
:03210100D0E032F9
:10262000E4FCFDFB7AC079A8F81204C07BE07A2EA6
:10263000790078001225DCC374129FF557E49EF5EB
:102640005690709BE0F55BF55AE4F558F559E5892D
:1026500054F04401F589758CFF758AFFC2B9D2A97F
:03266000D28C22F7
:0C2C090090709BE0F55AE4F558F5592254
:1024B100E5C520E3FB75C50775C50FE5C530E4FB30
:1024C100AFC6EF75F004A4FFAEF0E5C5C413135415
:1024D100037C002FF53CEC3EF53BE4F53AE53A256B
:1024E100E024B9F8A63B08A63CE53C2527F527E5FD
:1024F1003B3526F526053AE53AB40AE1E4F53922F9
:10187E00C0D075D00830160302197AE5C520E3FBF7
:10188E00E4F5C575C508F543754401E54364087074
:10189E0003021959E5C530E4FB85C62885C53DE52B
:1018AE00436407600EE5C520E3FBE54304F5C5443C
:1018BE0008F5C5E52875F004A4FFAEF0E53DC413A8
:1018CE001354037C002FF546EC3EF545E54325E029
:1018DE002429F8A64508A64690709AE05544606003
:1018EE00AF28122832AF3D122832E543B4060885E0
:1018FE0045418546428049E54364077043E53925F5
:10190E00E024BAF8C3E52796F527E5261896F526BE
:10191E00E53925E024B9F8A64508A646E54625276B
:10192E00F527E5453526F526FEAF277C007D0A1204
:10193E0004098E248F250539E539B40A03E4F539F7
:10194E000543E54425E0F544021899300F1EE4A244
:10195E00C492E4A2C592E5A29692E6A29792E725DA
:0F196E0060C4F53EAF3E122832853E40D0D022F5
:10210400C0D075D008300F659070A4E0FD7C0090BD
:1021140070ACE0FB24FFFFE434FFFE1203F5EF2470
:1021240001FFE43EFEC3E51F9FF51FE51E9EF51E5D
:102134008B3FE53F6021E51EF583E51FF582E0C492
:1021440054F02560C4F09070A4E0251FF51FE43519
:102154001EF51E153F80DB9070A4E024FFFFE434DD
:10216400FFFEC3E51F9FF51FE51E9EF51ED0D0227E
:0D2BFC00E4F56EF56FF570C2161227562233
:1023EE00C0D075D008E5606057201654122BA84057
:1023FE004F9070A4E025E09070E6F09070E6E060FB
:10240E003F20113C1228668F6D12002E056FE56F6E
:10241E007002056E7004E56E6480701CF56EF56FCB
:10242E000570E570B40C04D2168015122B95E5706C
:10243E0020E00512275680089070E6E014F080BB6D
:03244E00D0D022C9
:10294500E4907113F0A3F090710E120623000000BD
:102955000074FF78CDF608F6E4907115F0F561F591
:082965006090711274FFF02272
:10000E00C0D075D008756001C290122BFC7F021211
:05001E002C69D0D02286
:102B2A00C0D0C291E559240190710DF0E435589056
:062B3A00710CF0D0D02266
:102B4000C0D0C292E559240190710DF0E43558903F
:062B5000710CF0D0D02250
:10145500C0D075D008E49070E6F020C604E04401E1
:10146500F020C7079070E6E04402F0907112E0FFAB
:101475009070E6E0FE6F603BEE702590711BE0FF1B
:101485006005122C71802C90711AE0FF64036004D2
:10149500EFB40405122C71801A7F01122C69801398
:1014A5009070E6E030E0077F01122C7180057F0225
:1014B500122C719070E6E0907112F0300B1EA29420
:1014C500300C01B34016C218122C09907098E0FE3A
:1014D500A3E0FF12289A12000E02156820100302DD
:1014E5001568907096E0FEA3E0FFC3E54C9FFFE50D
:1014F5004B9EFED3E5429FE5419E4016D218907162
:101505000E12062300000000E4907113F0122C095E
:101515008051C21890710EE0F8A3E0F9A3E0FAA398
:10152500E0FBC3E542954CFFE541954BFE3395E065
:10153500FDFCEB2FFFEA3EFEE93DFDE83CFC90712A
:101545000E1206179070ACE0FF907113E004F06F77
:10155500701190709FE0FEA3E0FF12289A12000E12
:06156500122104D0D02287
:101F1500C0D075D00890710EE0F8A3E0F9A3E0FAFF
:101F2500A3E0FBC3E542954CFFE541954BFE339598
:101F3500E0FDFCEB2FFFEA3EFEE93DFDE83CFC90B1
:101F4500710E120617300E337F007E007D007C0077
:101F550090710EE0F8A3E0F9A3E0FAA3E0FBD31239
:101F650005DD4017907095E0FFD3E5599FE558943E
:101F7500004008122B2A7560028015300D129070F2
:101F8500AAE065597002E5587006122B2A75600A99
:031F9500D0D02287
:10224F00C0D075D00890710CE0FEA3E06559700303
:10225F00E5586E7002D291300E379070A2E0FEA357
:10226F00E0FFC3E54E9FFFE54D9EFEC3E5259FE5CD
:10227F00249E5007E4907114F080169070BDE0FF1B
:10228F00907114E004F06F7008122B40756003809A
:10229F0015300D129070ABE065597002E55870065D
:0922AF00122B4075600BD0D02207
:102A7600C0D075D00890710CE0FEA3E065597003D4
:0C2A8600E5586E7004D291D292D0D0229C
:101BE000C0D075D008E5607003021C6EE4F55C752A
:101BF0005F01E55C64086065E55C25E024ADF58285
:101C0000E43470F583E0FEA3E08E5DF55EF47003CE
:101C1000E55DF4603EE561555F7015E559655E7000
:101C200004E558655D7009E55F4261AF5C12254DC2
:101C3000E561555F601DE55E2401FFE4355DFEEF63
:101C400065597003EE6558700AE55FF45261AF5C48
:101C5000122595055CE55F25E0F55F8095C3E525D8
:101C600078CE96E52418965005A62408A625E560AA
:101C700014601614601814601A24F96011146013AB
:101C8000240B7012121455800D121F158008122299
:091C90004F8003122A76D0D02205
:10271D00CBEFCBEBFD7C007E407F00120409CDEBAF
:10272D00CD7C001203F58E1A8F1B74002FF582EEEF
:10273D003430AF82F5188F197E307F008E1C8F1DBF
:09274D008E1E8F1FD211C2122250
:10283200C211051FE51FAC1E7002051E14F5828C25
:1028420083EFF0E51F65197004E51E6518700675C3
:102852001E30751F00E51F651D7004E51E651C70A6
:0428620002D212226A
:10286600C212051DE51DAE1C7002051C14F5828EF4
:1028760083E0FFE51D65197004E51C651870067593
:102886001C30751D00E51F651D7004E51E651C7076
:0428960002D2112237
:10289A00C3E51F9FF51DE51E9EF51CC3E51D9400AB
:1028AA00E51C9430400BD3E51D9519E51C9518409D
:0E28BA000CE51B251DF51DE51A351CF51C222D
:101C990025732025627520256275202575202575F7
:101CA900202562752025627520256320256275200F
:101CB90025632025632025630D0A00632069676E6B
:101CC9002025752025752025752025752025752049
:101CD90025752025752025750D0A006320786D6905
:101CE9007420257520256275202562750D0A002A44
:101CF90056455253494F4E3A20522D44415320568E
:101D0900322E330D0A00632100632072646173006F
:101D1900632069676E006320786D697400633F0012
:101D290063006320007265736574002A4552524F3F
:101D3900523A20556E6B6E6F776E20636F6D6D61D1
:051D49006E640D0A00AC
:062C8700E4F578C21722FB
:100AD6009070E9EBF0A3EAF0A3E9F0300B13300CC9
:100AE600089071067401F0800D9071067402F08012
:100AF60005E4907106F09070E9E0FBA3E0FAA3E04C
:100B0600F91203BA643F6003020BAE9070ECE0F991
:100B1600A3E0FAA3E09070C1C9F0A3EAF0A3E9F05C
:100B260090709BE09070C4F090709AE09070C5F061
:100B3600907096E0FFA3E09070C6CFF0A3EFF09020
:100B460070A2E0FFA3E09070C8CFF0A3EFF0907022
:100B5600AAE09070CAF09070ABE09070CBF0300FC6
:100B6600047F3180027F309070CCEFF0907106E008
:100B76009070CDF03010047F3180027F309070CEBF
:100B8600EFF0300E047F3180027F309070CFEFF0AF
:100B9600300D047F3180027F309070D0EFF07BFF04
:100BA6007A1C79991200C9229070E9E0FBA3E0FA59
:100BB600A3E0F91203BAFF122B80500C9070EAE4FE
:100BC60075F00112049480E0E4907105F09070E9EC
:100BD600E0FBA3E0FAA3E0F912197D907105E02588
:100BE600E024EFF582E43470F583EEF0A3EFF090A5
:100BF60070E9E0FBA3E475F0011204AAA9F0FA1269
:100C060003BAFF122B8050E7907105E004F0E0B4C0
:100C16000BBB9070F0E090709BF09070F2E09070DB
:100C26009AF09070F3E0FFA3E0907096CFF0A3EFF8
:100C3600F09070F5E0FFA3E09070A2CFF0A3EFF084
:100C46009070F8E09070AAF09070FAE09070ABF0B7
:100C56009070FBE0FEA3E0FFEE4F24FF920FA3E0AF
:100C6600FEA3E0FFEE4F24FF920BEF64014E7003EC
:100C7600D38001C3920C9070FFE0FEA3E0FFEE4F1D
:100C860024FF9210A3E0FEA3E0FFEE4F24FF920E96
:0D0C9600A3E0FEA3E0FFEE4F24FF920D222D
:10177C009070E9EBF0A3EAF0A3E9F01203BA643F2E
:10178C0060030218137BFF7A1C79C49070ADE0FFE4
:10179C00A3E09070C1CFF0A3EFF09070AFE0FFA387
:1017AC00E09070C3CFF0A3EFF09070B1E0FFA3E036
:1017BC009070C5CFF0A3EFF09070B3E0FFA3E09072
:1017CC0070C7CFF0A3EFF09070B5E0FFA3E090707E
:1017DC00C9CFF0A3EFF09070B7E0FFA3E09070CB0F
:1017EC00CFF0A3EFF09070B9E0FFA3E09070CDCFF5
:1017FC00F0A3EFF09070BBE0FFA3E09070CFCFF0C0
:10180C00A3EFF01200C9229070E9E0FBA3E0FAA369
:10181C00E0F91203BAFF122B80500C9070EAE475B9
:10182C00F00112049480E0E49070ECF09070E9E028
:10183C00FBA3E0FAA3E0F912197D9070ECE025E02F
:10184C0024ADF582E43470F583EEF0A3EFF09070E4
:10185C00E9E0FBA3E475F0011204AAA9F0FA120363
:10186C00BAFF122B8050E79070ECE004F0E0B40863
:02187C00BB228D
:101B1C009070E9EBF0A3EAF0A3E9F01203BAB43F3A
:101B2C00297BFF7A1C79E490709CE0FFA3E0907015
:101B3C00C1CFF0A3EFF09070A9E09070C3F090705B
:101B4C009EE09070C4F01200C9229070E9E0FBA3F3
:101B5C00E0FAA3E0F91203BAFF122B80500C90703C
:101B6C00EAE475F00112049480E0E49070F2F090D5
:101B7C0070E9E0FBA3E0FAA3E0F912197D9070F292
:101B8C00E025E024ECF582E43470F583EEF0A3EF6D
:101B9C00F09070E9E0FBA3E475F0011204AAA9F03F
:101BAC00FA1203BAFF122B8050E79070F2E004F0A7
:101BBC00E0B403BB9070ECE0FFA3E090709CCFF01E
:101BCC00A3EFF09070EFE09070A9F09070F1E090BE
:041BDC00709EF022E5
:1006F9007B017A7079577D20122A929070ECEBF089
:10070900A3EAF0A3E9F04A70047F0180027F009018
:1007190070F9EFF0605F7B017A70795612156BC83A
:10072900ECC8C9EDC9CAEECACBEFCB9070A7E0FE01
:10073900A3E0FFE4FCFD1204C0C8ECC8C9EDC9CAB6
:10074900EECACBEFCB907098E0FEA3E0FFE4FCFD8E
:10075900EB2FFFEA3EFEED39FDEC38FC9070EF120D
:1007690006179070A7E0FEA3E0FFE4FCFD9070F38C
:1007790012061780767B017A70795612156BC8ECD0
:10078900C8C9EDC9CAEECACBEFCB9070A4E0FFE4AB
:10079900FCFDFE1204C0C8ECC8C9EDC9CAEECACB3B
:1007A900EFCB907098E0FEA3E0FFE4FCFDEB2FFF98
:1007B900EA3EFEED39FDEC38FC9070EF1206179019
:1007C90070ECE0FBA3E0FAA3E0F912156BC8ECC8E2
:1007D900C9EDC9CAEECACBEFCB9070A4E0FFE4FC27
:1007E900FDFE1204C09070F31206179070EFE0FC42
:1007F900A3E0FDA3E0FEA3E0FF780F1206048F70CB
:100809009070EFE0FCA3E0FDA3E0FEA3E0FFEE544F
:100819007FFEE48E6E8F6F122B959070F9E0600960
:10082900E49070F7F0A3F0800B1200269070F7EEB9
:10083900F0A3EFF0E49070E9F0A3F09070E9E0FE26
:10084900A3E0FFE4FCFD9070F3E0F8A3E0F9A3E076
:10085900FAA3E0FBC31205F3606C122C159070EB40
:10086900EFF09070F9E060149070EBE0FF9070F891
:10087900E02FF09070F7E03400F080189070F7E006
:10088900FEA3E0FF9070EBE0FD1220159070F7EEEB
:10089900F0A3EFF09070EBE0FF120003056FE56F36
:1008A9007002056E7004E56E64807009F56EF56F6F
:1008B9000570122B959070EAE004F070069070E9CB
:1008C900E004F00208449070F9E070139070F7E0CA
:1008D900FEA3E0FF122C809070F7EEF0A3EFF090EA
:1008E90070F7E0FF1200039070F8E0FF1200032296
:042CB7001229B32209
:0A2C39007BFF7A1C79F81200C92213
:10117F009070EC74FFF0A3741DF0A3740FF0A3E450
:10118F00F0A37402F07B017A707955122321EF706E
:10119F0004120FF8229070EC74FFF0A3741DF0A3EB
:1011AF007412F0A3E4F0A37406F07B017A70795502
:1011BF00122321EF70189070EC74FFF0A3741DF0E0
:1011CF00A37412F07B017A70795B120AD6229070A9
:1011DF00EC74FFF0A3741DF0A37419F0A3E4F0A353
:1011EF007405F07B017A707955122321EF700A7B19
:1011FF00017A70795A12177C229070EC74FFF0A369
:10120F00741DF0A3741FF0A3E4F0A37406F07B0128
:10121F007A707955122321EF700A7B017A70795B0E
:10122F00121B1C229070EC74FFF0A3741DF0A374BA
:10123F0026F0A3E4F0A37402F07B017A70795512C3
:10124F002321EF70189070EC74FFF0A3741DF0A3BE
:10125F007429F07B017A707956120AD6229070ECBD
:10126F0074FFF0A3741DF0A3742BF0A3E4F0A37428
:10127F0002F07B017A707955122321EF701890706C
:10128F00EC74FFF0A3741DF0A37429F07B017A7046
:10129F007956120AD622907055E0B464041206F9FA
:1012AF00229070EC74FFF0A3741DF0A3742EF0A3C2
:1012BF00E4F0A37405F07B017A707955122321EFC6
:1012CF007004122CB722907055E0B47604122C39AA
:1012DF0022907055E060097BFF7A1D79341200C9A6
:0112EF0022DC
:102AE30010170280FB7560047F01122C697F1E1290
:082AF3002BBB12117F80E922C8
:1027C800C0D0EF20E72CEF640A6027EF640D60119A
:1027D80074552578F582E43470F583EFF005788038
:1027E8001174552578F582E43470F583E4F0D21736
:0527F800F578D0D022AD
:1022B8002A4D4553534147453A2053746F72696E0E
:1022C8006720706172616D657465727320696E2034
:1022D800464C4153480D0A002A4D45535341474542
:1022E8003A2046696E69736865642073746F726911
:1022F8006E670D0A00000001C001C802000C001B37
:102308000100193C03FFFFFFFFFFFFFFFFFFFFFF77
:09231800FFFFFFFFFF00000003BE
:0A2C43007574227575FD1212F0225F
:1012F0009022FDE49324FF920BA3E49324FF920C2D
:10130000A3E49324FF9210A3E49390709AF09023A7
:1013100001E49324FF920FE49070A4F07F80EF60CB
:101320001490709AE05F60079070A4E02402F0EFE0
:10133000C313FF80E9300F069070A4E004F09023FF
:1013400002E49390709BF0902303E4939070A1F0DB
:10135000902304E493FF740193907096CFF0A3EF71
:10136000F0902306E493FF7401939070A2CFF0A352
:10137000EFF090709BE0FBFD7C007E037FE81204A1
:10138000099070A5EEF0A3EFF09070A4E0FA8BF056
:10139000A4FF9070A7E5F0F0A3EFF0EB1313543F18
:1013A0009070ACF0FB9070BDF0902308E49324FFA4
:1013B000920EA3E49324FF920DA3E4939070AAF0FD
:1013C00090230BE4939070ABF090230CE493907017
:1013D00095F09070A1E0FF7E009070A7E0FCA3E084
:1013E000FD1203F5907098EEF0A3EFF0EBFF7E0096
:1013F000EAFD7C001203F5E02F9070A0F090709849
:10140000E03E90709FF0E4FFEF25E0240DF582E4CC
:101410003423F583E493FC740193FDEF25E024ADC0
:10142000F582E43470F583ECF0A3EDF00FEFB4082F
:10143000D790231DE493FF74019390709CCFF0A389
:10144000EFF090231FE4939070A9F0902320E49391
:0514500090709EF022E7
:100FF800A20BE433857582857483F0A20CE433A3D5
:10100800F0A210E433857582857483A3A3F09070F1
:101018009AE0857582857483A3A3A3F0A20FE433B5
:10102800FFE5752404F582E43574F583EFF09070DC
:101038009BE0FFE5752405F582E43574F583EFF050
:101048009070A1E0FFE5752406F582E43574F58318
:10105800EFF0907096E0FEA3E0FFE5752407F582B7
:10106800E43574F583EEF0A3EFF09070A2E0FEA3F0
:10107800E0FFE5752409F582E43574F583EEF0A305
:10108800EFF0A20EE433FFE575240BF582E4357426
:10109800F583EFF0A20DE433FFE575240CF582E447
:1010A8003574F583EFF09070AAE0FFE575240DF52F
:1010B80082E43574F583EFF09070ABE0FFE57524BA
:1010C8000EF582E43574F583EFF0907095E0FFE556
:1010D80075240FF582E43574F583EFF0E49070E938
:1010E800F09070E9E0FF6408603BEF25E024ADF57F
:1010F80082E43470F583E0FEA3E0FFE5752410F583
:1011080082E43574F583C083C0829070E9E0D082B0
:10111800D08375F002120654EEF0A3EFF09070E958
:10112800E004F080BC90709CE0FEA3E0FFE575242D
:1011380020F582E43574F583EEF0A3EFF09070A902
:10114800E0FFE5752422F582E43574F583EFF0902D
:10115800709EE0FFE5752423F582E43574F583EF8E
:10116800F07BFF7A2279B81200C91227FD7BFF7A3B
:071178002279E01200C922F8
:10238800E5C520E3FB75C50675C50EE5C530E4FB5C
:10239800AFC6EF75F004A4FFE5C5C4131354037C5E
:1023A800002FFFEC35F0CF2401F548E43FF547F561
:1023B8004B85484CE5C520E3FB75C50775C50FE59A
:1023C800C530E4FBAFC6EF75F004A4FFAEF0E5C579
:1023D800C4131354037C002FF54AEC3EF549F54D20
:0623E800854A4ED21822C6
:1029D50030181D85474B85484CE5422401F548E4F0
:1029E5003541F54785494D854A4E85244985254A12
:0129F50022BF
:102AC900C21943878075985AE589540F4420F589BE
:0A2AD900758DFFD28ED2BCD2AC2264
:030023000228F3BD
:1028F300C0E0C0F0C083C082C0D075D0103098074C
:10290300AF99C2981227C8309904C299D219D0D06E
:09291300D082D083D0F0D0E03274
:080003008F993019FDC219228A
:082C61008F993019FDC2192200
:10291C00E5C520E3FB8FC5EF4408F5C5E5C530E4FC
:10292C00FBAFC6EF75F004A4FFAEF0E5C5C41313FE
:09293C005403FDE5F0EF4DFF220C
:1029B300E4F5A8F5E8F5B8F5F875700FE570A2E051
:1029C30092B5A2E192B3A2E292B4A2E392B202FF61
:0229D300FE22E2
:102B9500E570A2E092B5A2E192B3A2E292B4A2E3FB
:032BA50092B222C7
:0C2C1500E56E4480856F82F583E0FF22AD
:10002E0090D3557499F090ACAA7466F090D3557431
:10003E0090F0E56DF5F0E56ED2E7F583E56FF582AC
:0D004E00E5F0F0E0A2E730F701B340F72243
:10275600E570A2E092B5A2E192B3A2E292B4A2E33E
:1027660092B290D3557499F090ACAA7466F090D357
:10277600557480F090D3557499F090ACAA7466F0B5
:092786009080007414F0D21A22B4
:102BA800301A0D908000E020E703D38001C3921A09
:032BB800A21A223C
:1027FD0075700C122756122BA840FB75700D122BFD
:10280D0095E4F56EF56F856F82856E83E0F56D123B
:10281D00002E056FE56F7002056EE56F7004E56EB5
:05282D00648070E2224E
:032CC700C21A220C
:03005B000221E39C
:1021E300C0E0C0D0C2CC742D25C9F5C93013581531
:1021F3004FE54F7052E55570128551FCC2C0F55042
:10220300755501E55325E0F54F803CE555640170B4
:102213002375FCFFD2C00550E5506552700E301493
:1022230007F55585544F801FC213801B75550275E2
:102233004F028013E555B4020E8551FCC2C075559B
:0C22430001E55325E0F54FD0D0D0E0328B
:102AFB0075FCFFD2C075FE0B75518075EA0DC2FCDB
:082B0B00D2EC75540AC213223A
:10296D00C213A202921475FCFFD2C08F52E4F5552A
:10297D00CEEDCE8EFECEEBCE8E5385544FEF600254
:03298D00D2132240
:062C8D00D20212296D22A3
:062C9300C20212296D22AD
:082C69007D0B7B01122C8D2272
:082C71007D327B04122C8D2240
:102BBB00C21375FCFFD2C08F54E4F55585544FD228
:022BCB001322D3
:1008F9002A4D4553534147453A20615F7374203D62
:100909002025750D0A002A4D4553534147453A2084
:1009190061283029203D2025750D0A002A574152AA
:100929004E494E473A20416363656C65726174694B
:100939006F6E206F7574206F662072616E67653AFD
:1009490020615F73743D25752C2061303D2575202C
:1009590028672D7377697463682064697361626CB1
:100969006564290D0A002A4D4553534147453A20EC
:1009790070283029203D2025750D0A002A5741523B
:100989004E494E473A20507265737375726520253A
:1009990075206F7574206F662072616E6765205BC4
:1009A90025752C25755D0D0A002A5741524E494E71
:1009B900473A20427265616B776972652065727288
:1009C9006F722028425720747269676765722064C4
:1009D900697361626C6564290D0A002A5741524E98
:1009E900494E473A2049676E6974657220256264E9
:1009F90020636F6E666967757265643A20626F611C
:100A09007264206E6F7420666F756E640D0A002A19
:100A19005741524E494E473A2049676E697465728B
:100A29002025626420636F6E666967757265643A32
:100A3900206E6F20636F6E6E656374697669747971
:100A49000D0A002A5741524E494E473A20547261C5
:100A59006E736D697474657220636F6E666967750C
:100A69007265643A20626F617264206E6F742066E9
:100A79006F756E640D0A002A5741524E494E473A26
:100A89002044726F6775652069676E697465723A8B
:100A9900206E6F20636F6E6E656374697669747911
:100AA9000D0A002A5741524E494E473A204D616975
:100AB9006E2069676E697465723A206E6F20636F84
:0D0AC9006E6E65637469766974790D0A00BC
:072C7900EF60031F80FA2247
:102A5700A2029293E4F576F5777F78122C790577C1
:0F2A6700E57770020576E577640A457670EB2215
:100E6500E49070EEF09070E9F0A3F09070EDF0D2A0
:100E750002122A577F0612291C9070EAE02FF09083
:100E850070E9E03EF0C202122A579070EDE004F0DE
:100E9500E0B420DB9070E9E0FEA3E0FF7C007D205C
:100EA50012045E9070E9EEF0A3EFF07BFF7A08790B
:100EB500F99070C1EEF0A3EFF01200C9E49070EB69
:100EC500F0A3F0A3F07F0612291C9070ECE02FF040
:100ED5009070EBE03EF09070EDE004F0E0B420E5BA
:100EE5009070EBE0FEA3E0FF7C007D2012045E9095
:100EF50070EBEEF0A3EFF07BFF7A09790F9070C1EC
:100F0500EEF0A3EFF01200C99070EBE0FEA3E0FF56
:100F15009070E9E0FCA3E0FDC39FFFEC9EFEC3EFEC
:100F2500942DEE64809480502D7BFF7A097925906D
:100F350070C1ECF0A3EDF09070EBE0FFA3E09070D2
:100F4500C3CFF0A3EFF01200C97F06122C71C210B7
:100F55009070EE7406F0E49070E9F0A3F09070EDF7
:100F6500F07F0712291C9070EAE02FF09070E9E0FD
:100F75003EF09070EDE004F0E0B420E59070E9E01B
:100F8500FEA3E0FF7C007D2012045E9070E9EEF088
:100F9500A3EFF07BFF7A09796F9070C1EEF0A3EFB4
:100FA500F01200C99070E9E0FEA3E0FFC3947DEE66
:100FB50064809482400BD3EF94DBEE64809483408D
:100FC5002C7BFF7A0979859070C1EEF0A3EFF0A331
:100FD5007402F0A3747DF0A37403F0A374DBF01224
:100FE50000C97F05122C719070EE7405F09070EEBB
:030FF500E0FF22F8
:101A5500E49070E9F0300B1EA294300C01B34016EF
:101A65007BFF7A0979B21200C97F03122C71C20B70
:101A75009070E97403F0E49070EAF09070EAE0FF8A
:101A85006408606AEF25E024ADF582E43470F583DF
:101A9500E0FCA3E0F47002ECF4604B122C21401F33
:101AA5007F04122C717BFF7A0979E49070EAE004D7
:101AB5009070C1F01200C99070E97404F08027900D
:101AC50070EAE0FF122501401D7F04122C717BFF97
:101AD5007A0A79189070EAE0049070C1F01200C992
:101AE5009070E97404F09070EAE004F0808D9070D5
:101AF5009CE07002A3E06019122C9940147F041237
:101B05002C717BFF7A0A794C1200C99070E9740434
:071B1500F09070E9E0FF22EF
:10278F00D201121A5590711AEFF06002C201120EA7
:10279F006590711BEFF06002C20120C60B7BFF7AC0
:1027AF000A79801200C9C20120C70B7BFF7A0A7910
:0927BF00AC1200C9C201A2012202
:102B5600E4FF74162FF582E43471F58374FFF00FE9
:052B6600EFB404EE22B3
:0C2C2100EFC31325E02441FF122AAE226D
:102501009070EBEFF0E0FFC31325E02441FF7B0166
:102511007A7079ED9070F27401F01226639070EC8C
:10252100EFF09070EBE054012402FF74017E00C8CB
:10253100EFC8088005C333CE33CED8F9FF9070EDD4
:0C254100E0FDE4EF5D6003D38001C322E5
:10254D00CEEFCEEEC313FF2416F582E43471F5837E
:10255D00C083C082E0FDEE5401FC7401C8ECC808D4
:10256D008002C333D8FCF45DD082D083F0EF25E038
:10257D002440FFEEC3132416F582E43471AD82FCC2
:08258D007B01D2011226E222BB
:10259500CEEFCEEEC313FF2416F582E43471F58336
:1025A500C083C082E0FDEE5401FC7401C8ECC8088C
:1025B5008002C333D8FC4DD082D083F0EF25E024D0
:1025C50040FFEEC3132416F582E43471AD82FC7B23
:0725D50001D2011226E222EF
:10217400E4F571F572F57390709CE0FEA3E0FF4EF8
:10218400605C9070407404F0E4A3F0FCFD7BC0FA42
:10219400F9F81204C0C8ECC8C9EDC9CAEECACBEF3D
:1021A400CB7F007EC07DA87C001225DCEFF4049078
:1021B4007042F090709EE0FFC43354E0FF9070A929
:1021C400E024182F907043F07B017A7079407D04ED
:0F21D400122B6B7B017A7079407D04122B6B22EA
:062C99007F48122AAE2262
:101D4E009070E9EBF0A3EAF0A3E9F0907000EDFFDC
:101D5E007E017480F0A3E4F0C5827002158314C571
:101D6E0082C9C582C9CAC583CAE0F8A3C9C582C9DA
:101D7E00CAC583CAEEFBE8C313DBFCF5F0E045F001
:101D8E00F0A3E045F0F0A37407C39EFB6007E8C321
:101D9E0033DBFC8001E8D2E7F0A3C2E7F0C5827026
:101DAE0002158314C582BE0715A3A37480F0A3E4A5
:101DBE00F0C5827002158314C5827E0180010EDD8E
:101DCE00A0EF75F008A4240675F00784C333FF2234
:0C1DDE009070E9E4F0A3F0A3F0FDFF22F8
:102B6B00121D4ECEEFCE7F487C707D00CBEECBC2DC
:052B7B00011226E22218
:101E8100C0D075D00890709CE07002A3E07003028E
:101E91001F12740A2571F57190709BE06571707164
:101EA100F5719070407415F0A37401F0E572A3F020
:101EB100E573A3F0E56060080573E57370020572D0
:101EC100E529907044F0E52AA3F0E52BA3F0E52C79
:101ED100A3F0E52DA3F0E52EA3F0E52FA3F0E53067
:101EE100A3F0E531A3F0E532A3F0E533A3F0E53447
:101EF100A3F0E535A3F0E536A3F0E537A3F0E53827
:101F0100A3F0A3E540F07B017A7079407D15122B97
:041F11006BD0D0229F
:102A17000000CC01D8011400F0013C002800E401BB
:102A2700A0016C007800B40150009C0188014400AB
:050026007EFF7FFF22B8
:10201500CBEFCBCAEECAC9EDC9E9540FFFEAEB6FA6
:10202500540F25E0FFE433FE74172FF582EE342AB2
:10203500F583EAC4F854F0C868FEEBC4540F48FFB2
:10204500EE540FFEE4936EFA7401936FFBCFE9CF64
:10205500EFC4540F540FFFEAEF6B540F25E0FFE474
:1020650033FE74172FF582EE342AF583EAC4F8544B
:10207500F0C868FEEBC4540F48FFEE540FFEE4931E
:0C2085006EFA7401936FFBCEEACEFF22CE
:072C8000EEF4FEEFF4FF2269
:10245100FF2CBBFF2C4DFF2C57FF29F6FF2C9FFFB4
:102461002990FF2CA5FF2CBFFF2BEDFF2CABFF2AE2
:1024710037FF2B13FF2CC3FF2CCAFF2CCBFF2CCC17
:10248100FF2CCDFF2CCEFF2CCFFF2CD0FF2CD1FF6A
:102491002CD2FF2CD3FF2CD4FF2CD5FF2CD6FF2C14
:1024A100B1FF2CB1FF2CB1FF2CB1FF2CB1FF2CB12E
:0F2BDE00D296D29775D8C575DBECD2BDD2AD2299
:102AAE00E4F5678F65D21BD2DDFF1228C8EF6418DC
:0B2ABE006004EFB44003D38001C3228A
:1026E2009070E9ECF0A3EDF08C838D827879EBFEAB
:1026F2006006E0F6A308DEFA8B678F65D21BD2DD97
:1027020030010DCFEBCF1228C89070EBEFF08005AF
:0B271200E49070EBF09070EBE0FF2211
:102663009070EFEBF0A3EAF0A3E9F0CEEFCEA3E096
:10267300FFF5678E65D21BD2DD1228C8E4FE907089
:10268300F2E06E601D74792EF8E6FD9070EFE0FBCA
:10269300A3E0FAA3E0F98E82758300ED1203D30E53
:0326A30080DC22B6
:1028C800CEEFCEE4F562EE2402FDE433FCE5626D62
:1028D8007001EC6010756328D563FD201B03AF669B
:0B28E80022056280E175D8D57F002238
:042CBB0075D8D522D1
:0A2C4D008565DA75D8C5E4F5642248
:0A2C57008565DA75D8C5E4F564223E
:1029F600C0D075D010E567700775D8D5C21B800E9C
:102A0600AF64056474792FF8E6F5DA75D8C5D0D0C9
:012A1600229D
:062C9F0075D8D5C21B220E
:10299000C0D075D010E5646567700775D8D5C21BC7
:1029A000800EAF64056474792FF8E6F5DA75D8C542
:0329B000D0D02262
:062CA50075D8D5C21B2208
:042CBF0075D8E522BD
:0F2BED00E567700775D8D5C21B800375D8C52260
:062CAB0075D8D5C21B2202
:102A3700C0D075D010AF64056474792FF8A6DAE5B5
:102A4700646567700575D8C1800375D8C5D0D02275
:102B1300C0D075D010AF64056474792FF8A6DA7548
:072B2300D8D5C21BD0D0225F
:042CC30075D8D522C9
:012CCA0022E7
:012CCB0022E6
:012CCC0022E5
:012CCD0022E4
:012CCE0022E3
:012CCF0022E2
:012CD00022E1
:012CD10022E0
:012CD20022DF
:012CD30022DE
:012CD40022DD
:012CD50022DC
:012CD60022DB
:062CB10075D8D5C21B22FC
:03002B000226A604
:1026A600C0E0C0F0C083C082C0D075D01085D966A6
:1026B600E5D9131313541F75F003A42451F582E4CE
:1026C6003424F583E493740193FA740293F91206A1
:0C26D60060D0D0D082D083D0F0D0E032B1
:03000000022C2DA2
:0C2C2D00787FE4F6D8FD7581D0021F9876
:1003BA00BB010689828A83E0225002E722BBFE0241
:0903CA00E32289828A83E4932274
:1003D300F8BB010DE58229F582E5833AF583E8F060
:1003E300225006E92582C8F622BBFE05E92582C80C
:0203F300F222F4
:1003F500EFF88DF0A4FFEDC5F0CEA42EFEEC88F04D
:04040500A42EFE2201
:10040900BC000BBE0029EF8DF084FFADF022E4CCD7
:10041900F875F008EF2FFFEE33FEEC33FCEE9DECA0
:10042900984005FCEE9DFE0FD5F0E9E4CEFD22EDE6
:10043900F8F5F0EE8420D21CFEADF075F008EF2F30
:10044900FFED33FD4007985006D5F0F222C398FD21
:050459000FD5F0EA22BE
:10045E00C2D5EC30E709B2D5E4C39DFDE49CFCEEB9
:10046E0030E715B2D5E4C39FFFE49EFE120409C324
:10047E00E49DFDE49CFC800312040930D507C3E41F
:06048E009FFFE49EFE2228
:10049400C5F0F8A3E028F0C5F0F8E58215827002F3
:0604A4001583E038F02290
:1004AA00A3F8E0C5F025F0F0E58215827002158305
:0604BA00E0C838F0E82262
:1004C000E88FF0A4CC8BF0A42CFCE98EF0A42CFCDB
:1004D0008AF0EDA42CFCEA8EF0A4CDA8F08BF0A459
:1004E0002DCC3825F0FDE98FF0A42CCD35F0FCEBB8
:1004F0008EF0A4FEA9F0EB8FF0A4CFC5F02ECD397D
:0F050000FEE43CFCEAA42DCE35F0FDE43CFC22E9
:10050F0075F008758200EF2FFFEE33FECD33CDCCA3
:10051F0033CCC58233C5829BED9AEC99E582984026
:10052F000CF582EE9BFEED9AFDEC99FC0FD5F0D603
:10053F00E4CEFBE4CDFAE4CCF9A88222B800C1B92D
:10054F000059BA002DEC8BF084CFCECDFCE5F0CB6B
:10055F00F97818EF2FFFEE33FEED33FDEC33FCEBA4
:10056F0033FB10D703994004EB99FB0FD8E5E4F95F
:10057F00FA227818EF2FFFEE33FEED33FDEC33FC4C
:10058F00C933C910D7059BE99A4007EC9BFCE99A40
:10059F00F90FD8E0E4C9FAE4CCFB2275F010EF2F85
:1005AF00FFEE33FEED33FDCC33CCC833C810D70785
:1005BF009BEC9AE899400AED9BFDEC9AFCE899F8C0
:0E05CF000FD5F0DAE4CDFBE4CCFAE4C8F92253
:1025DC00C2D5E830E70FB2D5E4C39BFBE49AFAE42A
:1025EC0099F9E498F8EC30E717B2D51226121205D7
:1025FC004BE4C39BFBE49AFAE499F9E498F8800362
:10260C0012054B30D50DE4C39FFFE49EFEE49DFD07
:04261C00E49CFC221C
:1005DD00EB9FF5F0EA9E42F0E99D42F0EC6480C895
:0605ED0064809845F02235
:1005F300EB9FF5F0EA9E42F0E99D42F0E89C45F05E
:0106030022D4
:10060400E8600FECC313FCED13FDEE13FEEF13FFD4
:03061400D8F122F8
:0C061700ECF0A3EDF0A3EEF0A3EFF02256
:10062300A8828583F0D083D08212063A12063A124A
:10063300063A12063AE473E493A3C583C5F0C5836F
:10064300C8C582C8F0A3C583C5F0C583C8C582C821
:010653002284
:0C065400A42582F582E5F03583F58322B1
:060660008A838982E47325
:10005E00E56824C1F582E43470F583E005682290EA
:10006E0070BE3009039070C1E475F0011206B30240
:10007E0003BA2002E97F2ED2028018EF540F24908B
:10008E00D43440D4FF30060BEF24BFB41A00500313
:10009E002461FFE56960021569056CE56C70020567
:1000AE006B30090E9070BEE475F0011206B3EF02CC
:1000BE000693022C617403D2098003E4C209F56829
:1000CE009070BE1206CAE4F569F56BF56CE56960D1
:1000DE00077F201200A180F5F56AC203C202C20496
:1000EE00C205C207C208C20A12006DFF700D3009A8
:1000FE00057F001200B2AF6CAE6B22B42561C2D583
:10010E00C20612006DFF24D0B40A00501C75F00A0E
:10011E0020D50DC569A42569F5697002D20580E068
:10012E00C56AA4256AF56A80D724CFB41A00EF50A9
:10013E0004C2E5D2060202ACD20380C4D20280BE53
:10014E00D20480BAD2D580B8D20780B27F201200F6
:10015E00A12004077401B5690040F112005EFF1280
:10016E0000A10200DBD20AD208809312005EFB12BD
:10017E00005EFA12005EF94A4B700679787A037BBC
:10018E00FF200433E569602FAF6ABF00011F7E00B8
:10019E008E8275830012066660050EEE6F70F1C2D8
:1001AE00D5EBC0E0EAC0E0E9C0E0EE1202F0D0E02C
:1001BE00F9D0E0FAD0E0FB1203BAFF60A5EBC0E085
:1001CE00EAC0E0E9C0E01200A1D0E02401F9D0E0DD
:1001DE003400FAD0E0FBE56A60DDD56ADA80837B15
:1001EE00FF7A0279ECD2048098791080027908C2E5
:1001FE0008C20A8008D2D5790A8004790AC2D5E4E9
:10020E00FAFDFEFF12005EFC7B0820031312005E57
:10021E00FD7B1030020A12005EFE12005EFF7B2094
:10022E00EC3382D592D55013C3E43002069FFFE41F
:10023E009EFEE42003039DFDE49CFCE4CBF8C20388
:10024E00EC700CCFCECDCCE824F8F870F38017C349
:10025E00EF33FFEE33FEED33FDEC33FCEB33FB9966
:10026E004002FB0FD8E9EB300305F8D0E0C448B2EA
:10027E0003C0E00AEC4D4E4F78207B0070C2EAC0FE
:10028E00E01202F2D0F0D0E0200304C4C0E0C4B209
:10029E0003C0F012008AD0F0D5F0EB0200DB12069C
:1002AE00D301795301F758014A4C01464201FB4FE5
:1002BE00020344020349015F4302095501ED460161
:1002CE00ED4501ED47039B50014E2D01522E017558
:1002DE002B01562301732003862A0000016D3F3F38
:1002EE003F00790AA2D5200514300709B91002047F
:1002FE0004B9080104A2D5200802500104200466A6
:02030E00920457
:10031000B569005032C0E07F203005177F30A2045D
:1003200072087207500D120347C204C208C2077F49
:1003300030800F300703E9C0E01200A1300703D07E
:10034000E0F9D0E0B569CE3007177F30B9100C1254
:1003500000A17F583006077F788003B90803120098
:10036000A13004057F2D0200A17F20200AF87F2BF9
:100370002008F322920480CF286E756C6C29002D22
:1003800050434958D20312005E3003F8C203786923
:1003900030D504D202786AF602010C12005E240302
:1003A000B405004001E490037F93120092743A1266
:0A03B0000092D2057569040201F7FE
:102B8000EFC394094006EFC3940E4004EFB4200352
:052B9000D38001C32207
:102321009070E9EBF0A3EAF0A3E9F09070ECE0FB28
:10233100A3E0FAA3E0F91203BAFE9070E9E0FBA36F
:10234100E0FAA3E0F91203BAFD6E702AED600E9077
:1023510070EF74FFF5F012049445F070037F0022D2
:102361009070EAE475F0011204949070EDE475F058
:102371000112049480B5D3EE6480F8ED6480984036
:07238100037F01227FFF2210
:102A9200E94A4B7001221203BAFF6D700122EF70F6
:0C2AA20004FBFAF92209E970ED0A80EA51
:10156B009070FAEBF0A3EAF0A3E9F09070FAE0FBCD
:10157B00A3E0FAA3E0F91203BAFF122B80500C90F0
:10158B0070FBE475F00112049480E0D2019070FAC4
:10159B00E0FBA3E0FAA3E0F91203BAFF642B6004AB
:1015AB00EFB42D1D9070FAE0FBA3E475F00112046B
:1015BB00AAA9F0FA1203BA642D6003D38001C39277
:1015CB00019070FD120623000000009070FAE0FB02
:1015DB00A3E0FAA3E0F91203BAFF122BCD506A7FF6
:1015EB000A7E007D007C009070FDE0F8A3E0F9A37B
:1015FB00E0FAA3E0FB1204C0C8ECC8EDC0E0EEC0FB
:10160B00E0EFC0E09070FAE0FBA3E0FAA3E0F91280
:10161B0003BAFF3395E0FEEF24D0FFEE34FFFEE478
:10162B00FCFDD0E0FBD0E0FAD0E0F9EB2FFFEA3E77
:10163B00FEED39FDEC38FC9070FD1206179070FB37
:10164B00E475F00112049480823001109070FDE07B
:10165B00FCA3E0FDA3E0FEA3E0FF80119070FDE092
:0E166B00FCA3E0FDA3E0FEA3E0FF1206A52213
:10197D00907107EBF0A3EAF0A3E9F0907107E0FB9B
:10198D00A3E0FAA3E0F91203BAFF122B80500C90DA
:10199D007108E475F00112049480E0D20190710792
:1019AD00E0FBA3E0FAA3E0F91203BAFF642B600495
:1019BD00EFB42D1D907107E0FBA3E475F001120447
:1019CD00AAA9F0FA1203BA642D6003D38001C39261
:1019DD0001E490710AF0A3F0907107E0FBA3E0FA27
:1019ED00A3E0F91203BAFF122BCD503F907107E01F
:1019FD00FBA3E0FAA3E0F91203BAFF3395E0FEEF83
:101A0D0024D0FBEE34FFFA90710AE0FEA3E0FF7CD8
:101A1D00007D0A1203F5EF2BF0EE3A90710AF0906B
:101A2D007108E475F00112049480AD30010A9071D3
:101A3D000AE0FEA3E0FF800F90710AE0FEA3E0FF35
:081A4D00C3E49FFFE49EFE22AA
:10066600BB010CE58229F582E5833AF583E0225049
:1006760006E92582F8E622BBFE06E92582F8E22293
:0D068600E58229F582E5833AF583E49322AD
:10069300BB010689828A83F0225002F722BBFE0146
:0206A300F32240
:0E06A500C3E49FFFE49EFEE49DFDE49CFC2266
:1006B300F8E0FBA3A3E0F925F0F0E58215827002D0
:0706C3001583E0FA38F02274
:0906CA00EBF0A3EAF0A3E9F02231
:1006D300D083D082F8E4937012740193700DA3A3B6
:1006E30093F8740193F5828883E4737402936860CA
:0606F300EFA3A3A380DFCA
:102BCD00EFC394304009EFC3943A5003D38001C34F
:012BDD0022D5
:00000001FF
